:030000000219FDE5
:03000B000200AA46
:03002B0002019936
:03005B0002034F4E
:0300730002033550
:1000800002030406080C10182030406080040608A3
:100090000C10182030406080A0C000070F1F3F0DDB
:1000A0000D0403060D0503030202C2AF306308C24C
:1000B00063857C8AD2AF32C0D0C0E0206227E525BC
:1000C0006002E473E525F4C3334009758A00D26306
:1000D000F57C01D6F58A758B00758D00D262D0E073
:1000E000D0D0D2AF32C3E526334009758A00D2633F
:1000F000F57C01F6F58AC262E526F4603B306803C0
:10010000207213758B00758D00D0E0D0D0C292C2E2
:1001100094C296D2AF32C292C294C296206E0C2084
:100120006609740AD5E0FDE57E4290758B00758DF9
:1001300000D0E0D0D0D2AF32758A00D263757C0097
:10014000C28DD262212B01C4306805206602D29292
:1001500001C4306805206602D29401C430680520CD
:100160006602D29601C4C29330680A2066077408FA
:10017000D5E0FDD29201C4C29530680A20660774AA
:1001800008D5E0FDD29401C4C29730680A20660702
:100190007408D5E0FDD29601C4C2AFC2AD53E6EFFC
:1001A000C0D0C0E0D2D3D2AFE57D6009E57A60056A
:1001B000757A00413E757A01C2CEE52A6007207447
:1001C00049152A410A7800790020742EE580307E96
:1001D00001F430E60278FF53DACF207E0343DA20C1
:1001E000307E0343DA10C2D8C271E580307E01F45C
:1001F00030E60279FFC3E89970CB306103752A407D
:10020000207403752A40885FD27020740DE52B603E
:1002100004152B411A43DA01C2D8207002412DA8DF
:100220005F206102C270207402412B88227882B65E
:100230000403852224C3E52594404002D26420CFE4
:100240000AD0E0D0D043E610D2AD32C2CF053AE5B5
:100250007D6009E57B6005757B00612B757B01780E
:1002600002E52A6005307402152AC3E55F94014057
:10027000057562004187756300756C00E5622401B5
:10028000F56250037562FF7982B7020D306D1DC3B0
:10029000E52294324016854D227982B7030E306DE7
:1002A0000BC3E52294324004798E8722C3E523955F
:1002B0002260084004152341BB0523D8CA056CE51C
:1002C0006C7002156CD56D63756D017805C3E56CB6
:1002D000956E4057C3E56C956F50087801756D03B6
:1002E0000202EFC3E56C957050057801756D01C38E
:1002F000E5659524401E7982B704026120206D14C3
:10030000852465E56C046003856E6C756D0175234D
:100310003C02032BE5652850057565FF6120F565F6
:10032000E5650470067563FF756CFFD0E0D0D043BF
:10033000E610D2AD32C2AFC0D053E67FC260759135
:1003400000855694855795759104D0D0D2AF32C2AE
:10035000AF53E6EFC2ADC0D0C0E0C0F0D2D3D2AF51
:10036000A8FBA9FCE57D6007C3E913F9E813F8C20F
:10037000D830710261C153DACF207E0343DA1030E6
:100380007E0343DA20D271E580307E01F420E6025C
:10039000619888278928A1A053DACF207E0343DA09
:1003A00020307E0343DA10C2D8C271307402A18CAF
:1003B0007800E580307E01F430E602A18C885FA1F0
:1003C0007453DACF207E0343DA20307E0343DA1001
:1003D000C271206102819A53DACF207E0343DA1082
:1003E000307E0343DA20C2D8D271885A895BC3E8D1
:1003F0009558F8E99559F97B007E087A00C3E8948E
:100400008CE994005005755E00818C882178A2E605
:10041000A8216055C3E894C8E994005008E4D2E4E8
:10042000FB7A0A8167C3E89468E994015008E4D232
:10043000E3FB7A0F8167C3E894D0E994025008E4A3
:10044000D2E2FB7A1E8167C3E894A0E994055008C4
:10045000E4D2E1FB7A3C8167C3E89498E9940850C0
:1004600008E4D2E0FB7A787E00C3E8955CFCE9956D
:0F0470005DFD30E70AECF42401FCEDF43400FDEF
:10047F00755E00C3EC9AED9E5003755E01885C8932
:10048F005D855A58855B597802A174C3E89527F8A2
:10049F00E99528F9307C02A158307B02A158307AB7
:1004AF0002A15120750281BDE9FDE8FC81DCE9C3A1
:1004BF0013F9E813F8307902A151E9C313F9E813DE
:1004CF00F8307802A151E9C313FDE813FC2061262F
:1004DF00C3EC941CED9402400281F3ED7018C3EC51
:1004EF0094C850120529C3E529940A5002A18C75AE
:1004FF005F00D270A18CE529600215297400207F5E
:10050F00037896E624FAFEE43400FFC3EC9EFCED7C
:10051F009FFD500678007900A158C3EC94FFED942D
:10052F0000400678FF7900A158EC8575F0A4C5F05E
:10053F00A2F733F87900400302057478FF790002BF
:10054F000574E9C313F9E813F8307C0EE9600278FB
:10055F00FFC3E81338F8E43400F9C3E894FFE994D3
:10056F0000400278FF885FD270206102A18C741F57
:10057F00F4552F4BF52FC274EB7002D274752A40CD
:10058F00307403752A0A306102A1A020740353DA74
:10059F00FE207403752B20D0F0D0E0D0D0D2AD4325
:1005AF00E6103279010205D079030205D0790A02EB
:1005BF0005D0791E0205D079640205D079C80205ED
:1005CF00D07817E4D5E0FDD8FAD9F6227A147B78E3
:1005DF000205F77A107B8C0205F77A0D7BB40205C2
:1005EF00F77A0B7BC80205F77902B27DE4C295D585
:1005FF00E0FDD294D5E0FDC294D5E0FDD295D5E0D3
:10060F00FDD292E576D5E0FDC2927496D5E0FDD984
:10061F00D9EAF8D5E0FDD8FBDBCEC29522C37C002A
:10062F007D0075F00005F0EA33FAEB33FB50F6EB83
:10063F0013FBEA13FAC3E9FFE8FEE89AF8E99BF91E
:10064F005004EFF9EEF8B3EC33FCED33FDD5F0DFEA
:10065F00EDF9ECF822E889F08A20D2D4F8A9F07BE2
:10066F000030F70B7BFFF42401F8E9F43400F9E8CC
:10067F008520F0A4ADF0F8E98520F0A4AFF0FEEDF1
:10068F002EF974003FFA7C04C3EA13FAE913F9E870
:10069F0013F8DCF48BF030F70AE8F42401F8E9F4EE
:1006AF003400F9E889F0C2D4F8A9F0227882B604B0
:1006BF000302075AC3E55F9419401EE52D540670D7
:1006CF0018206D3678057994E7146007780A14605E
:1006DF00027812C3E54198401F306D098567657533
:1006EF006CFF756D01852224E4F545F546F547F558
:1006FF0048F549C26D02075AD26D7994E714701309
:10070F00E523F43333F913F8E9540104F9E854FEFF
:10071F0002074EE714147014E523F4333333F9133F
:10072F00F8E9540304F9E854FC020756E523F433BF
:10073F00333333F913F8E954070404F9E854F8C3D1
:10074F009440F8E99400F98845894622C3E541139E
:10075F00F9E54013F8C3E54598F8E54699F9500CCB
:10076F00C3E89480E994FF4016020792C3E8947F90
:10077F00E994005003020792787F7900020792787C
:10078F008079FF884A894B22E54A2547F8E54B35A2
:10079F0048F9854B20E4300701F43549FA30E70971
:1007AF00C3EA94F040150207D0C3EA940F50030236
:1007BF0007D078FF79FF7A0F0207D0780079007A97
:1007CF00F0C3E5249564500AC374019524500B02BD
:1007DF0007EEE54B20E70E0207EEE54B30E7068804
:1007EF004789488A492278A4E6FAC3E54A33F8E5EF
:1007FF004B33F9120664E930E70BC3E89480E994B0
:10080F00FF40130129C3E8947FE9940050020129A6
:10081F00787F79000129788079FFE820E715C3E513
:10082F002398F84009C3E894014003020850780167
:10083F00020850E8F424012523F8400302085078F9
:10084F00FF884C2278A5E6FAA848A949120664E960
:10085F0030E70CC3E89401E994FF4016020885C302
:0F086F00E894FFE99400500302088578FF7900B0
:10087E00020885780179FFE920E715C3E54C98F861
:10088E004009C3E8940140030208AC78010208ACA9
:10089E00E8F42401254CF840030208AC78FF8824C4
:1008AE002278FFC26420693D206A12D264C3E541FA
:1008BE00940A4009C3E52594405002C26479A1E729
:1008CE006023E541601F74FF8541F0848539F03067
:1008DE006A0375F005A4F8C5F0600278FFC3E895C9
:1008EE00675002A867886622C3E54094C8E5419424
:1008FE0000E5665003142107046002F56622788332
:10090E00E6F520120FCC75E8901205B275E890E569
:10091E00E820ECFBA8BDA9BE12106A757155757260
:10092E0000C3740013FD7455606613FC74552CFCE3
:10093E0074003DFDECFAEDFBC3E89AE99B4014E52B
:10094E00712455F571E5723400F572EA2CFAEB3D1F
:10095E00FB80E5AE71AF72C3E57213F9E57113F862
:10096E00C3E913F9E813F87A03C3E913F9E813F8A6
:10097E00DAF7AA201A700975710075720002099EC5
:10098E001AEA6008EE28FEEF39FFDAF88E718F72E0
:10099E002275E890227883E6FFE5E820ECF7A8BD03
:1009AE00A9BE0573C3E57394084052757300E9FA46
:1009BE0079A0E76044EA7007E574601B0209D9C3A9
:1009CE00E895746010E5745006600C140209E50495
:1009DE0060F90209E5E574F574C39472401B756401
:1009EE00C0C394044013756480C39404400B7564B3
:1009FE0040C39404400375640075BB0922EFC39491
:100A0E0001601F7455601BC3E894FFE994035012F4
:100A1E00C3E89571E995725009E564600C1564029E
:100A2E000A37E564F460020564A864C3E5249850AF
:100A3E0002A824C3E89565400AA865E565F460033D
:100A4E0085656488258826E573B4070375BB102277
:100A5E00743279A687F0A4C5F0A2F733F8C3E895EF
:100A6E00644002A864882288248825882688672204
:100A7E007540007541F022C2AF75C820A8CCA9CD33
:100A8E00AA3A30CF010A75C824D2AFC3EA13FAE9E5
:100A9E0013F9E813F8AB3BAC3C883B893CC3E89BAD
:100AAE00F8E99C20690A547FF930670261A8610554
:100ABE00AD3D8A3DF9EA9D547FFA600478FF79FFD7
:100ACE00AE3EAF3F8B3E8C3FC3EC9FFCC3E99CF523
:100ADE0042A83BA93CC3E89EF8E99FF9C3E5411340
:100AEE00FBE54013FAE82AF540E93BF5415006755F
:100AFE0040FF7541FF614FAA40AB41AC40AD417E16
:100B0E00047F02C3EB940440021E1FC3EB94084003
:100B1E00021E1FC3ED13FDEC13FCDEF7C3EA9CFAB5
:100B2E00EB9DFBEF6009C3E913F9E813F8DFF7EA71
:100B3E0028FAEB39FB8A408B4150067BFF8B408BAA
:100B4E0041C3EB94025002D2673069047F03617A8D
:100B5E007892E6FFC3E537948240110FC3E53794D0
:100B6E00A040010FC3EF940640027F057E02E541CF
:100B7E00C4540FF9E541C454F0F8E540C4540F28AD
:100B8E00F8C3E89EFAE99400FB4009C3EA9402EB2D
:100B9E00940050047A02E4FB61F4AA40AB41EBC42A
:100BAE00FEEAC4540F4EFCC3EA9CFAEB9400FBC35E
:100BBE00E813C313F8EA28FAEB3400FB8A408B41A2
:100BCE00C3EB94024002C2677802EBC4FE7B00EADC
:100BDE00C4540F4EFAC3EA98FA4005C39402500269
:100BEE007A027892E6FF30600261F48552568553A0
:100BFE0057D26043E680C3E49AF8E49BF9C3E83326
:100C0E00F8E933F93067028195E8FAE9FBD3E91385
:100C1E00FDE813FC88528953C3EF94036038EF202C
:100C2E00E00DE82CF8E93DF9ECFAEDFB020C50E88A
:100C3E0028F8E939F9C3E82402F8E93400F97AFE14
:100C4E007BFFC3EF9403400E8A548B55884E894F19
:100C5E008C508D5181C9885489558A4E8B4F8C503A
:0E0C6E008D51306920C3E53394034019E542EF
:100C7C00A2E713F8E555F4240138400B20E708757A
:100C8C0054FFF42401F55581C9E8FAD3E813FC8824
:100C9C0052C3EF94036020EF20E007E82CF8ECFA45
:100CAC0081B5E8282402F87AFEC3EF940340088A41
:100CBC0054884E8C5081C988548A4E8C50E56BC335
:100CCC00335002646BF56B30600281D3753404D2FF
:100CDC006043E680E52D5406601FA840A941C2AFD1
:100CEC0053E67F759100C3E498F594E499F59575F6
:100CFC009104D26043E680D2AF22D2657544007570
:100D0C002000306B03752040020D25D26575440020
:100D1C00752040306B03752000D2AF78012067221C
:100D2C00E52D54066002C265C3E541940540137875
:100D3C000294054008780394054002780630690255
:100D4C00780A206019E544601530690AC3E53394CC
:100D5C00034003D53406D2AFD26CC10791DBD2AFBE
:100D6C000000C2AF20672AE541C3FB940F40027B11
:100D7C000FEB240530730123306A027428206201C2
:100D8C0023F93069027982E58D13E58B13C3994001
:100D9C00B10544E59B5440B52002A1F130690A0825
:100DAC00C3E8940A400108A14E206502A125C26542
:100DBC0053E67F7591003067107594007595FC753E
:100DCC009104D26043E680A125AE40AF41C3EE331F
:100DDC00FEEF33FF50047EFF7FFFC3E49EF594E4E7
:100DEC009FF595A1CBC3E53394025002A125306544
:100DFC0002A125D802C105A14EC26C53E67F7591A4
:100E0C0000855494855595759104854E56854F579C
:100E1C00D26043E680D2AFE52D54066008206A020A
:100E2C000533020E41306C0D206B0A2065071581CD
:100E3C0015810216CA2278003064053065027801EB
:100E4C00E53775F007A4F9E5F028F5F0E9A2F01301
:100E5C00A2F113A2F213F537C394785003753778C7
:100E6C00C3E53795384008D266C292C294C2963018
:100E7C006002C17B855056855157D26043E6802273
:100E8C00D287207D11C2AF754302C295D293D2AFE7
:100E9C00759F80021067C2AF754302C295D297D27C
:100EAC00AF759F80021067C287307243207D20C2CD
:100EBC00AF754303900177757E20C296C29730625E
:100ECC0004D294C1D3D295D2AF759F89021067C258
:100EDC00AF754303900177757E20C292C293306246
:100EEC0004D294C1F3D295D2AF759F8102106720C2
:100EFC007D17C2AF754303900152C296306202D285
:100F0C0094D2AF759F89021067C2AF7543039001ED
:100F1C0052C292306202D294D2AF759F8102106796
:100F2C00D287207D11C2AF754304C293D297D2AF42
:100F3C00759F81021067C2AF754304C297D293D2DA
:100F4C00AF759F89021067C287307243207D20C223
:100F5C00AF754305900166757E08C294C2953062E8
:100F6C0004D292E173D293D2AF759F80021067C204
:100F7C00AF754305900188757E80C294C29530622E
:100F8C0004D296E193D297D2AF759F80021067205E
:100F9C007D17C2AF754305900148C294306202D2EE
:100FAC0092D2AF759F80021067C2AF754305900156
:100FBC005CC2943062EBD296D2AF759F8002106700
:100FCC00D287207D11C2AF754306C297D295D2AF9E
:100FDC00759F89021067C2AF754306C293D295D232
:100FEC00AF759F81021067C287307242207D20C28C
:100FFC00AF754301900188757E80C292C2933062B6
:10100C0004D2960113D297D2AF759F81021067C29A
:10101C00AF754301900166757E08C296C297306227
:10102C0004D2920133D293D2AF759F890167207D90
:10103C0016C2AF75430190015CC292306202D29627
:10104C00D2AF759F810167C2AF754301900148C251
:10105C0096306202D292D2AF759F89C266229001FD
:0E106C0046757E00C292C294C296C293C2958F
:10107A00C297C26222788076070876070876010846
:10108A0076040876FF0876FF08760908760208765D
:10109A0001087601788C76010876000876B408761D
:1010AA00FF0876FF0876FF0876030876FF087601C0
:1010BA000876FF0876250876D00876780876C80874
:1010CA0076040876FF08760108760008767A0876AC
:1010DA000A0876010876010876000876FF227887E2
:1010EA00E6FFC272BF0302D2727888C27DE630E19F
:1010FA0002D27DC27E7889E630E102D27EC3EF94C5
:10110A00026008758E01D27302111A758E00C273BD
:10111A00227880E6149000809378A4F67881E61409
:10112A009000809378A5F67886E61490008D9378DF
:10113A00A6F6789FE6F8700108C3E8941140027891
:10114A0011E82828F56E256E256E28F56F256E287C
:10115A0028F570789CE67538FF75390CB402067567
:10116A0038A075390AB4030675388275390578A32B
:10117A00E61490009A93F569116A22C2A4C2A07873
:10118A009DE6B40104D2A4C2A0B40204C2A4D2A0AF
:10119A00227896E6FA7897E6FB7888E6B40305C3E0
:1011AA00EB940EFB307F047A007BFFC3EB9AFCC3FF
:1011BA00948250027C827575000575EC8575F0A4E1
:1011CA00C3E5F0947D40F222D27F319B1205C17AA9
:1011DA00007B007C101205B7E55F2AFA74003BFB1E
:1011EA00DCF37C04C3EB13FBEA13FADCF7FEC27FE1
:1011FA00319B22E5EF20E6037520000520903FFF92
:10120A00E520146006901FFF1460009304600375C4
:10121A00EF1253D9BF7581C043FF801205B275EF33
:10122A000243B203E5B3240420E70DF521E5E320E8
:10123A00E0068521B343E301116A7580FF75A48036
:10124A0075F1F075D4BF75900275A5FC75F2FD7540
:10125A00D50275A61175A0EE75F3F175E241E4F8B1
:10126A00F6D8FD756B01117F121719789886767575
:10127A003001C2AF1205CB1205DB1205C11205E21D
:10128A001205C11205E91205C112183B1205CB124B
:10129A0005CB1205C6C2AF78FA79FA308607D9FBB0
:1012AA00D8F7021C0011E8311B3185319B789886EA
:1012BA0076116A75B68075A900757D0075885075B6
:1012CA00891275C82475910475D84075A82275B815
:1012DA000275E690759B80759D0075D10E75BC5898
:1012EA0075BB0975BA1175E8801205B2D2AF120939
:1012FA000C53DACF207E0343DA20307E0343DA1020
:10130A0043DA01C2D8C2711205CBD2617B037A0CCF
:10131A00E55E70077A0CDB0302129F1205C120708A
:10132A000302129FC270E55FC3940240E1E52F54A5
:10133A001F856160F561B560D5DAD5C26153DACF30
:10134A00207E0343DA20307E0343DA10C2D8C2710A
:10135A0078A2E67008D274E52F54E0F52FC27575AD
:10136A0029001205C6307409C3E529940A4002D23D
:10137A00751205B778023074027800C3E55F9840A9
:10138A00F0C2AF1205DB1205DB1205DBD2AF120584
:10139A00CB754D001205B7788CE6C3940150030251
:1013AA001474E530C394015003021474207435C3D5
:1013BA00E55F94FF5003021474C2AF1205F0D2AF76
:1013CA001205C6C3E55F940150EFC2AF1205DB12E6
:1013DA0005BC1205DBD2AF1205C6C3E55F94FF4018
:1013EA00E90218C07F05D27F319B1205C6C2AFC27F
:1013FA007F319BAE5FC3E55F947FD2AF4076120523
:10140A00B2C2AF1205F0D2AFDFDC31D2C3EE94051F
:10141A007897F61205CB12175A1218437F0AD27F11
:10142A00319B1205C6C2AFC27F319BAE5FC3E55F77
:10143A00947FD2AF50E61205B2C2AF1205DB120595
:10144A00BC1205DBD2AFDFD631D2EE24057896F690
:10145A001205CB12175A1218721205C6319BC3E530
:0F146A005F94FF500261B60218C0C3E55F954D55
:101479004003855F4D1205C678017988E7B40302F8
:101489007805C3E55F984002619EC2AF1205F0126C
:1014990005F01205F0D2AF1205CB753000E4F53135
:1014A900F5320531E531F470390532789AE6781963
:1014B900146012783214600D787D14600878FA147B
:1014C9006003753200C3E53298401715327531B49F
:1014D90078998676C2AF1205F0D2AF7898867612DF
:1014E90005C61205BCE52A7005307402419F7801D2
:1014F9002074027806C3E55F9840A71205C6E52A5D
:10150900700302129FC2AF116AE4F522F523F52494
:10151900F525F526F56AD2AF7885E6C333F568E493
:10152900F545F546F547F548F549F573F52CF52DDB
:10153900F53775730875BB101205B212099FE5E8F6
:1015490020ECFBA8BDA9BEE97001F888741209A3B3
:1015590075730875BB107887E6FE760211E87887FF
:10156900EEF6C2AF7564FF120A5E852264852265B4
:10157900852266D2AF75220175240175250175266C
:101589000185636C756D0175B69075A903757D014B
:101599007888E6B40307C27D307602D27DD268D25C
:1015A90069753300120FCC120FF3120A7E120A85E5
:1015B900120A7E120A85120A7E0215D1C2AF11E8FB
:1015C900D2AF75730075BB09120D171206BB120E47
:1015D90042120E8C120A85120D06306D0312075B3A
:1015E9002067031208AF3067031208F6120E421281
:1015F9000EB3120A85120D17306D03120797120EDA
:1016090042120F2C120A85120D06306D031207F5CE
:10161900120E42120F53120A85120D17306D031262
:101629000853120E42120FCC120A8512099F120D8D
:1016390006120E42120FF31209A3120A8530692FFE
:10164900206B2C85676485676585636C756D017989
:10165900187A0CC3E533994009C269D26A8A3502FE
:101669001678C3E55F940140030215D10216D23002
:101679006A1B206B18E535147004C26AA1C5F535DB
:10168900C3E55F940140030215D10216D2753600F5
:10169900C3E5629401400985676585636C756D01D1
:1016A900C3E56278FA985021307404E52A601A7803
:1016B900F0306B058567647820C3E541985002A135
:1016C900D10536E55F6002C1D5753600C2AF116A32
:1016D9007887E6FE760211E87887EEF6E4F522F5DA
:1016E90023F524F525F526F568C26875B68075A930
:1016F90000757D00D2AF1205B2116A307406E52A71
:101709007002419F788DE6C394014002617B81A6F6
:10171900901A0D782012179CE520B4A50CA3121776
:101729009CE520B45A0302173A117F12175A02177F
:1017390059901A0378807B0A12179CA308DBF99049
:101749001A0F788C7B1812179CA308DBF9901A27BB
:1017590022C2AF1217DB1217B5901A00740E1217B6
:10176900A1A374041217A1A374141217A1901A0348
:1017790078807B0A1217A0A308DBF9901A0F788CDE
:101789007B181217A0A308DBF91217EE1217CC90D9
:101799001A2722E493F622E6438F01538FFD75EF52
:1017A9000275B7A575B7F1F0538FFE22438F024337
:1017B9008F0175EF0275B7A575B7F1901A0DF05342
:1017C9008FFC22901A0D74A5F1A1901A0E745AF18A
:1017D900A1227A3079D07820901A40F19CE520F73F
:1017E90009A3DAF7227A3079D0901A40E7F1A109F2
:1017F900A3DAF922AB77A878BB01027980BB020290
:101809007981BB03027982BB04027994BB05027911
:1018190083BB06027986BB07027992BB08027987E6
:10182900BB0902799CBB0A027988BB0B027989E85A
:10183900F7227C051205CBDCFB22C2AF1205DB12B5
:1018490005E21205E91205F01205BC1205DB1205C5
:10185900E21205E91205F01205BC1205DB1205E2D8
:0E1869001205E91205F0D2AF22C2AF1205F04F
:101877001205E91205E21205DB1205BC1205F0128A
:1018870005E91205E21205DB1205BC1205F0120587
:10189700E91205E21205DBD2AF22AE77AF78C2AF0D
:1018A7001205DB1205DB1205DB1205BCDEF21205A1
:1018B700F01205BCDFF8D2AF221143113B113B7583
:1018C700770175780175790011A17C05AD5F120567
:1018D700CBC3ED955F70F5C3E55F9401400AC3E59F
:1018E7005F94FF40340218FE1217FD12175A114376
:1018F700C2AF75EF12113BDCD30579C3E5799403C9
:10190700500280C4113B0578E5771490009F93F847
:1019170008C3E57898500280AC113B113B0577C3AB
:10192700E577940C5002809A12107F12175AC2AFB3
:0519370075EF12113BE9
:0319FD000211FDD7
:101A00000E041407070104FFFF09020101A55A0192
:101A100000B4FFFFFF03FF01FF25D078C804FF01DA
:081A200000FF0A010100FFFFB5
:101A400023506C6174696E756D3530417633232097
:101A500023424C48454C492346333930232020202B
:101A60002020202020202020202020202020202076
:101C0000C2AFC2D353D9BF7581C043B20343FF8073
:101C1000752438752503B1C975EF0275E24043F1AB
:101C20004053A4BF75D400D2867DFA780379E67C50
:101C300010752200752300901DD67B0675249875BB
:101C400025013086028142208608D8FBD9F9DCF7CD
:101C500081B4308608D8FBD9F9DCF781B4B189E4C6
:101C600093A3C39A6004DDC381B4DBDBB17B600264
:101C7000812B7B08E493FAA3B15CDBF87A30B15C8A
:101C8000752200752300B17BEAFCEBFDC3ED94FEE9
:101C9000400EB17B8A278B28ED30E0048A828B834B
:101CA000B17B7AC270D8C3ED94FE601350CEBD00F4
:101CB00025EC60097520007521FF0200008100A855
:101CC00027A9280809D804D90281D3B17FEA89AAB3
:101CD000F281C50D81A0C3ED94035049EDA2E092BD
:101CE000007AC5C3E5829400E583941C50902000DF
:101CF00010438F02438F0175B7A575B7F1F030001F
:101D00001FA827A9280809438F01538FFDD804D99C
:101D100002A12089AAE275B7A575B7F1F0A3A10DBC
:101D2000538FFC817C7AC1BD030CE493A3FAB140CC
:101D3000DCF8B138817C817EAA22AB23B15CEBFA5E
:101D4000EA6222752608C3E52313F523E52213F57D
:101D50002250066323A0632201D526EAB1C9B1C986
:101D600075260AEAF4200102D286300102C286B149
:101D7000C9C3134002C201D526EB22B17FEAFB2082
:101D80008602A17F308602A184752608AE24AF2585
:101D9000C3EF13FFEE13FEB1CDB1C9C3EA13308612
:101DA000024480FA30E703632201C3E52313F523DD
:101DB000E52213F52250066323A0632201D526D91C
:101DC000E52265236523F52222AE24AF250E0FDE22
:101DD000FEDFFCD20122424C48656C693437316326
:041DE000F390060175
:00000001FF
